:1000000000308A0025280234A00003088301A700DD
:100010000408A8000A08A9008A012A08AC002B08D5
:10002000AD000B198B1E1728831252200B1183125F
:100030002C08AA002D08AB002808840029088A0093
:1000400027088300A00E200E0900A101A201A30130
:10005000A4010030AB000330AA0025308400263014
:1000600036208316FF23900083017428A6004120C8
:100070008000840A04082606031D372800348312F2
:10008000AA00AB1B4A282B088A002A08AA0A0319CF
:10009000AB0A820083132B1883172A08AA0A84004C
:1000A000000808008312A30183128F206328023006
:1000B00025020318692810306128A508031969284A
:1000C0002030A3006928220803195728013A031990
:1000D0005D28A5080319A11F6E28A3012308850028
:1000E0000130A206A10A0800FF2383169000CF303A
:1000F00083168500831285018316990107308312C8
:100100009900810182308316810051309F000130B7
:1001100083129F009F148B160B118B178E2883124E
:100120009F1808001E08A4009F1489302402031899
:100130009B28A50108008F3024020318A228A501DE
:0A014000A50A08000230A50008001F
:02400E00843FED
:00000001FF
